:1000000029C0000042C0000040C000003EC0000007
:1000100099C000003AC0000038C0000036C000009F
:100020005AC0000032C0000030C000002EC00000E6
:100030002CC000002AC0000028C0000026C000001C
:1000400024C0000022C0000020C000001EC000002C
:100050001CC0000011241FBECFE5D4E0DEBFCDBF21
:1000600010E0A0E6B0E0E0EDF6E002C005900D92F1
:10007000AE38B107D9F710E0AEE8B0E001C01D928C
:10008000A73CB107E1F72BD121C3BACF10928F0063
:100090008CB59DB59093C2008093C1008091BA0049
:1000A0009091BB00A091BC00B091BD008093C300B3
:1000B0009093C400A093C500B093C60080918F00B8
:1000C000882321F708958091BE008F3F19F084BDE9
:1000D00087E085BD08951F920F920FB60F921124ED
:1000E0008F939F93AF93BF938091BA009091BB0081
:1000F000A091BC00B091BD000196A11DB11D8093DF
:10010000BA009093BB00A093BC00B093BD00809157
:100110008F008F5F80938F00BF91AF919F918F91E0
:100120000F900FBE0F901F901895982F80917F0011
:10013000882321F088B39095892302C088B3892B46
:1001400088BBC1CF1F920F920FB60F9211248F93CD
:1001500080918E0085BB80917F0088BB15BC8F91FC
:100160000F900FBE0F901F9018955D9BFECF8CB91E
:1001700008950F931F93CF93DF93062FEC0110E0A8
:1001800003C08991F2DF1F5F1017D8F3DF91CF9181
:100190001F910F910895CF93DF93E7DFC1ECD0E07B
:1001A0008D81E3DF219780E0CB3BD807C9F7DF9152
:1001B000CF910895FC012091BF003091C000809143
:1001C000C1009091C200280F391F31832083809194
:1001D000900090919100AC0160E070E08091C300CC
:1001E0009091C400A091C500B091C600480F591F5E
:1001F0006A1F7B1F42835383648375838091C10090
:100200009091C2002817390740F44F5F5F4F6F4F3E
:100210007F4F4283538364837583089510928F00C8
:100220005F9904C080918F008230D0F380918F005D
:10023000089582E990E060EE70E046E050E016D26A
:10024000809193008F3FB1F488EF8093920082E019
:10025000809393001092940084EB80939500109209
:1002600096001092970082E990E060EE70E046E020
:1002700050E00CD2809192008093BE0010928E00CC
:1002800010927F0090919300292F90FF03C08FEF71
:1002900080938E0021FF03C08FEF80937F008091B9
:1002A0008E0085BB80917F0088BB9874946B92BB55
:1002B0009091950080E020919400820F911D909381
:1002C000C0008093BF009091970080E0209196003D
:1002D000820F911D9093910080939000089584B7B0
:1002E000806884BF84B7806884BF8FE78BBB88E455
:1002F00081BB8FEF84BB87BB9CDF10BC83E089B9D7
:1003000088E18AB982E08EBD15BC789489B784648F
:1003100089BFAA248824992493945F9BE6C08CB15A
:10032000893521F4B3DE89E536DFF7CF813059F422
:1003300075DF823090F79CB180918E00811190958D
:1003400095BBC1DEEACF8F3319F40FDF8A2D10C0C1
:10035000883541F480E690E065E10BDF88248394E2
:100360009924DBCF8837B1F2853421F4FEDE892D64
:10037000FCDED3CF882021F4823411F4E3C5CDCF45
:10038000873409F069C01BBA87B986E886B989B78E
:100390008F7B89BF82E085BD86E790E068E0E9DE7B
:1003A000C0E0D1E05F9BFECF8CB1823031F58FEFA2
:1003B00084BD8E01EE24FF241CC084B58823E9F798
:1003C000369A3699FECF84B1D0DE85B190E00F2CFD
:1003D00002C0880F991F0A94E2F7E82A22E0F20E81
:1003E00038E0F31621F48E2DC0DEEE24FF240150F8
:1003F00010400115110509F7D5CF8E3671F40EDFC7
:10040000823018F48CB1D82FC0E008DF823050F66B
:100410008CB190E0C82BD92BC5CF833439F4FEDEE4
:10042000823008F0BFCF8CB187B9BCCF863439F4A5
:10043000F5DE823008F0B6CF8CB185BDB3CF823502
:1004400019F08FE392DEAECF16B889B7806489BF0A
:1004500015BC8FE78BBB61CF853639F4DFDE823088
:1004600008F05BCF9CB085E683CF803129F5D6DEDE
:10047000823008F052CFFCB0D1DE823008F04DCF90
:100480000CB110E00AC0CADE823030F48CB1E12F2A
:10049000F0E0EE56FF4F80831F5F1017A0F382E954
:1004A00090E06F2D70E0402F50E0F0D08FED8F1571
:1004B00008F033CFBEDE31CF813109F02ECFAEDE72
:1004C000823008F02ACF0CB1A9DE823008F025CFA7
:1004D0001CB182E990E0602F70E0412F50E0C6D05F
:1004E00082E990E0612F45DE18CF99B380B3809503
:1004F00030EBB32EB82290959F77B92A82958074FD
:10050000B82ABA1409F409CFC1DD24E0C22ED12CD7
:10051000C1E0D0E08E010C2C02C0000F111F0A9424
:10052000E2F7402F502F5B21252F30E08A2D90E0FD
:10053000802391232817390751F1552331F1A02A3F
:100540009EEFE92E9FEFF92EEC0CFD1C892D90E01B
:100550000E2C02C0959587950A94E2F780FF17C08C
:10056000802FE3DD02C0CC0FDD1FEA94E2F7FE012D
:10057000E0959E22882031F0F601EB57FF4F8081F5
:100580000ADE05C0802FF1DD02C04095A422089448
:10059000C11CD11CF8E0CF16D10409F0B9CF82EA12
:1005A000E82E80E0F82E00E010E02091C3003091AA
:1005B000C4004091C5005091C600602FF7018281B0
:1005C0009381A481B581281739074A075B0708F48E
:1005D00042C0281739074A075B0749F42091C10038
:1005E0003091C2008081918128173907A0F1C1E0C4
:1005F000D0E002C0CC0FDD1F6A95E2F74C2F5C2FD4
:100600005B21252F30E08A2D90E08C239D23281735
:10061000390709F1552369F0AC2AC701CBDD90FEFB
:100620001AC08C2F82DD8820A1F0F801EB57FF4F14
:100630000DC04095A422C701BDDD91FE0CC08C2FDA
:1006400074DD882031F0F801E058FF4F8081A3DD90
:1006500002C08C2F8ADD0F5F1F4F26E030E0E20ED4
:10066000F31E0430110509F0A0CF57CEDC01CB01F9
:10067000FC01E199FECF06C0FFBBEEBBE09A3196CC
:100680000DB20D9241505040B8F70895DC01A40F0F
:10069000B51F4150504040F0CB01840F951F2E9163
:1006A00005D041505040D8F70895262FE199FECF4C
:1006B0009FBB8EBBE09A01970DB2021631F02DBBA5
:1006C0000FB6F894E29AE19A0FBE0895F894FFCF1E
:1006D000555354435254424F582C393231363030EE
:1006E0002C76362E31005254426F7841444300FF3D
:0E06F00032343638003133353761303962002C
:00000001FF
